:0300000002403B80
:0C403B00787FE4F6D8FD758121024082F8
:1045EF00901E5BA3E0FAA3E0F5828A83E4FF122218
:0945FF00BD1244ED12295180FBAC
:1044B80047616D65204F7665722100426C61636BC0
:1044C80020436865737320566963746F727921009D
:1044D8005768697465204368657373205669637407
:0544E8006F7279210054
:0A43AB00421EA00007421EA20007F8
:1037CB00901DCDE4F0A374EFF0A374BCF0A3744090
:1037DB00F07B177A01E4FDFC7F28FE123F10E4FF1B
:1037EB00FE124645901DCFE4F0A374EBF07B137AE9
:1037FB00017D047C007F2C7E00123CBE901DCFE42B
:10380B00F0A374ECF07B147A017D037C007F2B7E9C
:10381B0000123CBE901DCFE4F0A374E8F07B107A4D
:10382B00017D077C007F2F7E00123CBE901DC5E4FE
:10383B00F0A304F0901DC5E0FEA3E0FFC3940FEED0
:10384B006480948050347C007D0F122040EF24075D
:10385B00FDE43EFC901DE4F0A3EDF0E4A3F0A3F037
:10386B007B107A017F2FFE122E0B901DC6E004F009
:10387B0070C2901DC5E004F080BA901DC5E4F0A3A2
:10388B0004F0901DC5E0FEA3E0FFC3940FEE64802F
:10389B009480503D7C007D0F122040AC06AD07EDAF
:1038AB00242FFFE43CFEED242FFBE43CFA901DE4B7
:1038BB00E4F0A374E8F0E4A3F0A3F07D07FC122E70
:1038CB000B901DC6E004F070B9901DC5E004F080AC
:0138DB00B13B
:0138DC0022C9
:0A3BCD00901DC2EDF0901DC1EFF055
:103BD700D3940E4003023CBDE0FFC39400500302A0
:103BE7003CBDA3E0FED3940E4003023CBDEEC3945C
:103BF700005003023CBDEF75F00FA4FF901EA4E038
:103C0700FBA3E0FAA3E02FF9EA35F0FA901DC2E032
:103C17007E0029F9EE3AFA1220156003023CBD90A6
:103C27001EA7E0FEA3E0FF7C007D02122052ED4CB0
:103C37007002800274FF901DC3F0A3F0901DC1E0D5
:103C470075F00FA42436FFE435F0AD07FCA3E0754B
:103C5700F00FA4240EFFE435F0AB07AE04AF05FC6C
:103C6700AD03A3E0FBA3E0901DD3CBF0A3EBF0A340
:103C77007401F07B067A001217C3901EA8E004F0C7
:103C87007006901EA7E004F0901EA7A3E0FD901D0C
:103C9700C1E075F00FA4FF901EA4E0FBA3E0FAA318
:103CA700E02FF9EA35F0FA901DC2E07E0029F9EE1F
:063CB7003AFAED12202E86
:013CBD0022E4
:0A3FA800901DCAEDF0901DC9EFF066
:103FB200D3940E400302403AE0FFC394004079A339
:103FC200E0FED3940E5071EEC39400406BEF75F097
:103FD2000FA4FF901EA4E0FBA3E0FAA3E02FF9EAEE
:103FE20035F0FA901DCAE07E0029F9EE3AFA122065
:103FF200157045901DCB74BCF0A37440F0901DC9A0
:10400200E075F00FA42436FFE435F0AD07FCA3E021
:1040120075F00FA4240EFFE435F0AB07AE04AF0534
:10402200FCAD03901DD374BCF0A37440F0A37401E3
:08403200F07B067A001217C3AF
:01403A002263
:1042A100EF75F00FA4242FFEE435F0901DC5F0A3A7
:1042B100CEF0ED75F00FA42407FEE435F0A3F0A3D2
:1042C100CEF07FE07EFF124645901DC5E0FAA3E0E7
:1042D100FBFFAE02C006C007A3E0FCA3E0FDEB2498
:1042E1000FFBE43AFA901DC7E0FEA3E0240FFFE4C0
:0F42F1003E901DCFF0A3EFF0D007D006023CBEE9
:0A423900901EA0A3E0FFA3A3E0FD88
:10424300EF75F00FA4242FFEE435F0901DC1F0A309
:10425300CEF0ED75F00FA42407FEE435F0A3F0A330
:10426300CEF0E4FFFE124645901DC1E0FAA3E0FB49
:10427300FFAE02C006C007A3E0FCA3E0FDEB240FE2
:10428300FBE43AFA901DC3E0FEA3E0240FFFE43EF3
:0E429300901DCFF0A3EFF0D007D006023CBE86
:0731CC00F074FFA3F0A3F073
:1031D300901DC7EFF0A3ECF0A3EDF0A3EAF0A3EB8F
:1031E300F0E4901EA9F0A3F0901DCCE0FEA3E0FF55
:1031F300901DC9E02FF0901DC8E03EF0901DCEE079
:10320300FEA3E0FF901DCBE02FF0901DCAE03EF03F
:10321300901DC8E0FEA3E0FFC3EE64809480405796
:10322300D3EF940EEE64809480504CA3E0FEA3E0B1
:10323300FFC3EE64809480403ED3EF940EEE64802F
:103243009480400302337D901DC8E0FEA3E0FF7C21
:10325300007D0F122040901EA4E0FBA3E0FAA3E040
:103263002FF9EA3EFA901DCAE0FEA3E029F9EA3EEF
:10327300FA122015FD700302337DED75F002121F63
:10328300F3AFF0901DC7E06F600302337D901DCC58
:10329300E0FEA3E0FF64014E7008A3E07002A3E028
:1032A3006010BEFF1EBFFF1B901DCEE07002A3E0A7
:1032B3007011901EAAE004F07042901EA9E004F081
:1032C3000231EB901DCCE07002A3E0700C901DCE98
:1032D300E07004A3E064016015901DCCE0FEA3E060
:1032E300FF4E701BA3E0B4FF16A3E0B4FF11901EC2
:1032F300AAE004F07006901EA9E004F00231EBEF9F
:1033030064014E700C901DCEE07004A3E064016074
:1033130016901DCCE0B4FF20A3E0B4FF1BA3E0B4E0
:10332300FF16A3E0B4FF11901EAAE004F07006900C
:103333001EA9E004F00231EB901DCCE0FEA3E0FFF8
:1033430064014E700AA3E0F47003A3E0F4601AEF83
:10335300F47002EEF460030231EB901DCEE07004D2
:10336300A3E0640160030231EB901EAAE004F07055
:1033730006901EA9E004F00231EB901EA9E0FEA323
:03338300E0FF2246
:102FF900901DC3ECF0A3EDF0901DC1EEF0A3EFF02E
:10300900E4901DC5F0A3F0FC7D0F122040901EA492
:10301900E0FBA3E0FAA3E02FF9EA3EFA901DC3E032
:10302900FEA3E029F9EA3EFA122015FF75F0021213
:103039001FF3AFF0EF3395E0901DC5F0A3EFF090CB
:103049001DC1E0FCA3E0FDA3E0FAA3E0FB901DCCC9
:10305900E4F0A304F0E41231CFC006C007901DC507
:10306900A3E0FF901DC1E0FCA3E0FDA3E0FAA3E00B
:10307900FB74FF901DCCF0A3F0E41231CFD0E02F08
:10308900FFD0E03ECF2401FDE43FFCC3ED9405EC05
:103099006480948040037F0122901DC5A3E0FF90C6
:1030A9001DC1E0FCA3E0FDA3E0FAA3E0FBE4901D51
:1030B900CCF0A31231CCC006C007901DC5A3E0FF18
:1030C900901DC1E0FCA3E0FDA3E0FAA3E0FBE490BE
:1030D9001DCCF0A3F0A3F0A304F01231D3D0E02F5C
:1030E900FFD0E03ECF2401FDE43FFCC3ED9405ECA5
:1030F9006480948040037F0122901DC5A3E0FF9066
:103109001DC1E0FCA3E0FDA3E0FAA3E0FB901DCC08
:10311900E4F0A3041231CCC006C007901DC5A3E09A
:10312900FF901DC1E0FCA3E0FDA3E0FAA3E0FB745E
:10313900FF901DCCF0A3F0A3E4F0A304F01231D367
:10314900D0E02FFFD0E03ECF2401FDE43FFCC3EDEA
:103159009405EC6480948040037F0122901DC5A3EF
:10316900E0FF901DC1E0FCA3E0FDA3E0FAA3E0FBB2
:1031790074FF901DCCF0A3F01231CFC006C00790A8
:103189001DC5A3E0FF901DC1E0FCA3E0FDA3E0FA8B
:10319900A3E0FB901DCCE4F0A304F0A3E4F0A304A6
:1031A900F01231D3D0E02FFFD0E03ECF2401FDE46F
:1031B9003FFEC3ED9405EE6480948040037F0122B5
:0231C9007F0085
:0131CB0022E1
:1045B3007E007C00122FF9EF60037F0222901EA77A
:0F45C300E07004A3E064E170037F01227F002217
:1039E100901EA7E07002A3E07003023AD7E4901D95
:1039F100C1F0A3F0E4901DC3F0A3F0901DC1E0FE5F
:103A0100A3E0FF7C007D0F122040901EA4E0FBA3E9
:103A1100E0FAA3E02FF9EA3EFA901DC3E0FEA3E02D
:103A210029F9EA3EFA122015FF3395E0FE901EA710
:103A3100E0B50625A3E0B50720901DC1E0FFA3E096
:103A4100901DC5CFF0A3EFF0901DC3E0FFA3E09060
:103A51001DC7CFF0A3EFF0801A901DC4E004F070F1
:103A610006901DC3E004F0901DC3E07004A3E06460
:103A71000F7088901DC2E004F07006901DC1E00433
:103A8100F0901DC1E07004A3E0640F60030239F5FA
:103A9100901DC5E0FEA3E0FF7C007D0F1220409049
:103AA1001EA4E0FBA3E0FAA3E02FF9EA3EFA901D81
:103AB100C7E0FCA3E0FD29F9EA3CFAE412202E90CC
:103AC1001EA8E024FFF0901EA7E034FFF0901DC572
:063AD100A3E0FF123FA874
:013AD70022CC
:1040C700E4901EA7F0A3F0901DC1F0A3F0E4901DAB
:1040D700C3F0A3F0901DC1E0FEA3E0FF7C007D0FBD
:1040E700122040901EA4E0FBA3E0FAA3E02FF9EA18
:1040F7003EFA901DC3E0FEA3E029F9EA3EFAE41276
:10410700202E901DC4E004F07006901DC3E004F05B
:10411700901DC3E07004A3E0640F70B8901DC2E067
:1041270004F07006901DC1E004F0901DC1E070041A
:10413700A3E0640F70971237CB7D077F070242A178
:1044ED00E4901EA7F0A3F0901DC1122288000000D9
:1044FD000FE4FF1241C0901EA4EBF0A3EAF0A3E974
:10450D00F0E4FFFE1243591237CB7D077F070242BD
:01451D00A1FC
:1029510012456FEF24417003022BA024E0700302A3
:102961002B8424F07003022A3D24F87003022A020A
:1029710024FC605D24FE6030146003022BAB124521
:102981006FEF64FE60F8124239901EA3E024FFF05D
:10299100901EA2E034FFF0C3E0648094805030E4E4
:1029A100F0A3740EF0022A3012456FEF64FD60F857
:1029B100124239901EA1E024FFF0901EA0E034FFE6
:1029C100F0C3E0648094805006E4F0A3740EF080BC
:1029D1005E12456FEF64FB60F8124239901EA1E070
:1029E10004F07006901EA0E004F0C3901EA1E094D4
:1029F1000F901EA0E0648094804004E4F0A3F08076
:102A01002E12456FEF64F760F8124239901EA3E071
:102A110004F07006901EA2E004F0C3901EA3E0949F
:102A21000F901EA2E0648094804004E4F0A3F09033
:102A31001EA0A3E0FFA3A3E0FD0242A112456FEF98
:102A410064EF60F8901EA0A3E0FFA3A3E0FD123B9A
:102A5100CD901EA0A3E0FFA3A3E0FD1245B3901DFE
:102A6100C0EFF0901DC0E07003022BAB7F007EF839
:102A7100124645901DC0E024FE6052046003022B03
:102A810069901DCDE4F0A3747EF074FFA3F0A3F070
:102A91007B047A017D5A7C007F3C7E00123F1090BE
:102AA1001DC7E4F0A37410F0A374FFF0A37444F005
:102AB100A374B8F0A37410F0A37401F07B40FA7D05
:102AC100647C007F647E00123386022B63901DCDEF
:102AD100E4F0A3747EF074FFA3F0A3F07B047A0109
:102AE1007D5A7C007F3C7E00123F10901EA0E0FECC
:102AF100A3E0FF7C007D0F122040901EA4E0FBA309
:102B0100E0FAA3E02FF9EA3EFA901EA2E0FEA3E06C
:102B110029F9EA3EFA122015FF75F002121FF3AFF0
:102B2100F0EF901DC76013E4F0A37410F0A374FFDD
:102B3100F0A37444F0A374C38011E4F0A37410F003
:102B4100A374FFF0A37444F0A374D8F0A37410F03D
:102B5100A37401F07B40FA7D647C007F507E0012FB
:102B61003386901DC07403F0E4FFFE124645124502
:102B71006FEF64DF6003022A6412456FEF64DF6068
:102B8100F8800812456FEF64DF60F81240C7901EAD
:102B9100A0E4F0A37407F0A3E4F0A37407F02212F9
:0A2BA100456FEF64BF60F81239E1E0
:012BAB002207
:1043B500441E6C000000E0441E6800000020441EFE
:1043C5005700001C004D1E5BFF3E6CFF3AD80100F4
:0543D50000011C0000C6
:10430000901E8EEBF0A3EAF0A3E9F0901E87E0F98F
:10431000A3E0FAA3E0901E91C9F0A3EAF0A3E9F0AC
:10432000901E8A74FF122249EC4D4E4F602A901E57
:1043300091E0FBA3E475F00112209EA9F0FA12208F
:1043400015FF901E8EE0FBA3E475F00112209EA9DC
:08435000F0FAEF12202E80C8E4
:014358002242
:05447E00901DC4EDF0EB
:10448300901DC9EBF0A3EAF0A3E9F0901DC574FFFA
:10449300122249EC4D4E4F601B901DC4E0FF901D4E
:1044A300C9E0FBA3E475F00112209EA9F0FAEF1214
:0444B300202E80D760
:0144B70022E2
:103E6C00901DC0EFF0E0FF75F003A42464F582E42C
:103E7C00341EF583E0FBA3E0FAA3E0F9C003C00213
:103E8C00C001EF25E025E0246CF582E4341EF583B7
:103E9C00E0FCA3E0FDA3E0FEA3E0FFE47B02FAF963
:103EAC00F8122119901DC512227CD001D002D0032A
:103EBC00E4FD12447E901DC0E0FF75F003A4246164
:103ECC00F582E4341EF583E0FBA3E0FAA3E0F9EFFE
:103EDC0025E025E02457F582E4341EF583E0FCA3AD
:103EEC00E0FDA3E0FEA3E0FF901DC512227CE4FDE3
:103EFC0012447E901DC0E02467F582E4341EF583E5
:043F0C007401F0222A
:053AD800901DC0EFF09D
:103ADD00A312228800000000901DC512228800004C
:103AED000000901DC0E025E025E0246CF582E43453
:103AFD001EF583E0FCA3E0FDA3E0FEA3E0FF901D17
:103B0D00C5E0F8A3E0F9A3E0FAA3E0FBC312223667
:103B1D005077E47F02FEFDFC901DC5E0F8A3A3A342
:103B2D00E0122119901DC0E075F003A42464F58204
:103B3D00E4341EF583E0FBA3E0FAA3E0F98F828E57
:103B4D00831220B445F0601F901DC1E0FCA3E0FD81
:103B5D00A3E0FEA3E02401FFE43EFEE43DFDE43CD2
:103B6D00FC901DC112227C901DC5E0FCA3E0FDA3BD
:103B7D00E0FEA3E02401FFE43EFEE43DFDE43CFC59
:103B8D00901DC512227C023AEFE47F64FEFDFC908D
:103B9D001DC1E0F8A3E0F9A3E0FAA3E0FB1221199F
:103BAD00901DC0E025E025E0246CF582E4341EF57F
:0F3BBD0083E0F8A3E0F9A3E0FAA3E0FB1221A450
:013BCC0022D6
:0526EC00901DC9EFF094
:1026F100901DCE12228800000000E4901DD4F0A3AA
:10270100F0901DC9E0FF2467F582E4341EF583E0F3
:10271100700F901E5BA3E0FAA3E0F5828A83122278
:10272100BDE4FFFEFDFC901DCAE0F8A3E0F9A3E0C3
:10273100FAA3E0FBC3122236700302294A901DC995
:10274100E025E025E02468F582E4341EF583E0F815
:10275100A3E0F9A3E0FAA3E0FB901DCAE0FCA3E02B
:10276100FDA3E0FEA3E0FF1221A4901DD2EEF0A391
:10277100EFF0901DC9E025E025E02468F582E434FE
:102781001EF583E0F8A3E0F9A3E0FAA3E0FB901DB6
:10279100CAE0FCA3E0FDA3E0FEA3E0FF1221A4AC8C
:1027A10000AD01AE02AF03EC4D4E4F600E901DD354
:1027B100E004F07006901DD2E004F0901DC9E02500
:1027C100E025E0246CF582E4341EF583E0FCA3E00F
:1027D100FDA3E0FEA3E0022932901DCEE0FCEC3324
:1027E100500302294AE47F02FEFDFC901DCEE0F871
:1027F100A3E0F9A3E0FAA3E0FB122119901DC9E0BF
:1028010075F003A42464F582E4341EF583E0FBA390
:10281100E0FAA3E0F98F828E831220B445F07010A4
:10282100901DD5E004F0700F901DD4E004F08007F6
:10283100E4901DD4F0A3F0901DD2E0FEA3E0FFA32D
:10284100E06E7003A3E06F6003022923901DD6128E
:10285100228800000000901DD2E0FEA3E0FFE4FC0E
:10286100FD901DD6E0F8A3E0F9A3E0FAA3E0FBC3D5
:1028710012223640030228F6901DD2E0FEA3E0FFAB
:10288100C007C006901DCEE0FCA3E0FDA3E0FEA3BF
:10289100E0FF901DD6E0F8A3A3A3E02FFFEA3EFEE0
:1028A100E93DFDE83CFCE47B02FAF9F812211990BC
:1028B1001DC9E075F003A42464F582E4341EF58398
:1028C100E0FBA3E0FAA3E0F98F828E83D0E0D0F0A1
:1028D1001220EC901DD6E0FCA3E0FDA3E0FEA3E0F6
:1028E1002401FFE43EFEE43DFDE43CFC901DD612D4
:1028F100227C022857901DCEE0FCA3E0FDA3E0FE60
:10290100A3E0FF901DC9E025E025E02468F582E4FD
:10291100341EF583E0F8A3E0F9A3E0FAA3E0FB029B
:102921002119901DCEE0FCA3E0FDA3E0FEA3E0FF92
:10293100EF24FFFFEE34FFFEED34FFFDEC34FFFC2E
:0F294100901DCE12227C0227DA74FFFFFEFDFCF0
:012950002264
:05369900901EABEFF0F4
:10369E00E0FF2467F582E4341EF583E07012901E7D
:1036AE005BA3E0FAA3E0F5828A831222BD7F01229A
:1036BE00901EABE025E025E02457F582E4341EF59C
:1036CE0083E0FCA3E0FDA3E0FEA3E0FF901EACE0D0
:1036DE00F8A3E0F9A3E0FAA3E0FBC31222364003FD
:0336EE000237C8D8
:1036F100901EABE025E025E02468F582E4341EF558
:1037010083E0F8A3E0F9A3E0FAA3E0FB901EACE0AC
:10371100FCA3E0FDA3E0FEA3E0FF1221A4901EB2F2
:10372100EEF0A3EFF0901EABE075F003A42464F576
:1037310082E4341EF583E0FBA3E0FAA3E0F9901ED6
:10374100B3E025E0FF901EB2E0338F82F5831220B3
:10375100B4FF901EB4E5F0F0A3EFF0E4901EB0F0DA
:10376100A3F0901EB4E0FEA3E0FF901EB0E0FCA326
:10377100E0FDC39FEE6480F8EC6480985046901E93
:10378100B3E02DFF901EB2E03CFEEF25E0FFEE33EB
:10379100FE901EABE075F003A42464F582E4341EB0
:1037A100F583E0FBA3E0FAA3E0F98F828E83E4F5D1
:1037B100F01220EC901EB1E004F07006901EB0E013
:0737C10004F0809E7F00224E
:0237C8007F027E
:0137CA0022DC
:0E414700901EC0EFF0A3EBF0A3EAF0A3E9F0A6
:104155004A6067901EC0E075F003A42461F582E40F
:10416500341EF583E0FBA3E0FAA3E0FFAE02AD0346
:104175007C00A804C005C006C007901EC1E0FBA3D3
:10418500E0FAA3E0AE02AD03D003D002D001C39B99
:10419500FFEE9AFEED99FDEC98FCA312227C901E91
:1041A500C4E0FCA3E0FDA3E0FEA3E0FF901EAC127B
:0A41B500227C901EC0E0FF12369934
:0141BF0022DD
:0541C000901DC0EFF0AE
:1041C500C007A3E0FCA3E0FDA3E0FEA3E0FF901D74
:1041D500CA12227CD0071226EC901DC512227C74CF
:1041E500FFFFFEFDFC901DC5E0F8A3E0F9A3E0FA92
:1041F500A3E0FBC31222367004FBFAF922901DC01E
:10420500E075F003A42461F582E4341EF583E0FB38
:10421500A3E0FAA3E0FFAE02AD03901DC5A3E0F94C
:10422500A3E0FAA3E02FFFEA3EFEE93DFDA907AAB8
:0342350006AB05D0
:014238002263
:0E38DD00901E94EFF0A3EBF0A3EAF0A3E9F045
:1038EB00A3E0FCA3E0FDA3E0FEA3E0FF901DCA1242
:1038FB00227C901E94E0FF1226EC901E9C12227CE0
:10390B0074FFFFFEFDFC901E9CE0F8A3E0F9A3E022
:10391B00FAA3E0FBC31222367004FBFAF922901EC5
:10392B0094E075F003A42461F582E4341EF583E082
:10393B00FBA3E0FAA3E0FFAE02AD037C00901E9C5C
:10394B00E0F8A3E0F9A3E0FAA3E02FFFEA3EFEE9DB
:10395B003DFDEC38A907AA06AB05C002C001901EBD
:10396B0095E0F9A3E0FAA3E0901E87C9F0A3EAF073
:10397B00A3E9F0901E98E0FCA3E0FDA3E0FEA3E01A
:10398B00FF901E8A12227CD001D002124300901E9F
:10399B0094E0FFA3E0FBA3E0FAA3E0F91241479008
:1039AB001E94E075F003A42461F582E4341EF583C4
:1039BB00E0FBA3E0FAA3E0FFAE02AD03901E9CA3D5
:1039CB00E0F9A3E0FAA3E02FFFEA3EFEE93DFDA9F3
:0539DB0007AA06AB0580
:0139E00022C4
:1000030000000000000000000000000000000000ED
:100013003F400000000000000000300040003000BE
:100023004000000009000BC03D000BC03D0009006B
:1000330018C024407FE0224031800000180024C013
:100043001B000D803240018003801C4027401C8030
:1000530007400040100060000000000000000000A6
:100063000000000000001F802040402000004020CE
:1000730020401F8000000000090006001F800600CA
:1000830009000000040004003F8004000400000095
:1000930000100060000000000000000004000400E5
:1000A3000400040004000000000000400000000001
:1000B30000000000002001C00600380040000000DE
:1000C3001F802040204020401F800000000010407F
:1000D3003FC000400000000018C0214022402440DF
:1000E3001840000010802040244024401B80000062
:1000F30002000D0011003FC0014000003C8024407D
:1001030024402440238000001F80244024403440A6
:10011300038000003000200027C0380020000000CA
:100123001B802440244024401B8000001C0022C06C
:10013300224022401F800000000000000840000011
:100143000000000000000000046000000000000048
:10015300000004000A00110020804040090009004B
:100163000900090009000000000040402080110040
:100173000A00040018002000234024001800000097
:100183001F802040274029401F400000004007C037
:1001930039000F0001C0004020403FC024402440EC
:1001A3001B8000001F802040204020403080000042
:1001B30020403FC0204020401F80000020403FC01F
:1001C30024402E4030C0000020403FC024402E0079
:1001D300300000000F0010802040224033800200D6
:1001E30020403FC0040004003FC020402040204086
:1001F3003FC02040204000000060202020203FC05E
:100203002000200020403FC024400B0030C020408D
:1002130020403FC020400040004000C03FC03C00A1
:1002230003C03C003FC0000020403FC00C402300FF
:100233003FC020001F802040204020401F8000003E
:1002430020403FC024402400180000001F802140AC
:10025300214020E01FA0000020403FC02440260092
:1002630019C0004018C024402440224031800000BF
:10027300300020403FC020403000000020003F807D
:10028300004000403F80200020003E0001C00700E6
:1002930038002000380007C03C0007C038000000C9
:1002A300204039C0060039C02040000020003840FB
:1002B30007C0384020000000304021C026403840AD
:1002C30020C00000000000007FE04020402000002C
:1002D300000070000C00038000400000000040207C
:1002E30040207FE0000000000000200040002000CC
:1002F300000000000010001000100010001000109B
:100303000000000040000000000000000000028028
:100313000540054003C0004020003FC004400440A6
:1003230003800000000003800440044006400000F6
:1003330000000380044024403FC0004000000380CD
:100343000540054003400000000004401FC0244056
:1003530024402000000002E0055005500650042010
:1003630020403FC00440040003C00040000004409C
:1003730027C000400000000000100010041027E018
:100383000000000020403FC00140070004C00440BB
:10039300204020403FC000400040000007C0040050
:1003A30007C0040003C00000044007C00440040069
:1003B30003C00040000003800440044003800000A9
:1003C300041007F004500440038000000000038081
:1003D3000440045007F00010044007C0024004002A
:1003E30004000000000006400540054004C0000072
:1003F300000004001F800440004000000400078048
:100403000040044007C000400400070004C001800E
:1004130006000400060001C0070001C0060000003A
:10042300044006C0010006C0044000000410071089
:1004330004E00180060004000000044005C00640FB
:10044300044000000000000004007BE040200000A6
:10045300000000000000FFF000000000000040204A
:100463007BE004000000000040008000400020000A
:100473002000400000000000000000000000000019
:10048300000000000000000000001FCC000C000072
:100493000000000000000800300060000800300089
:1004A30060000000022003FC1E20022003FC1E202B
:1004B3000220000000000E1811043FFF10840C7886
:1004C300000000000F0010840F3800C00778188464
:1004D3000078000000780F8410C411240E9800E403
:1004E300008400080800680070000000000000009D
:1004F3000000000000000000000007E018182004BE
:1005030040020000000040022004181807E0000029
:10051300000000000240024001800FF00180024011
:10052300024000000080008000800FF800800080FF
:10053300008000000001000D000E0000000000001C
:100543000000000000000080008000800080008028
:10055300008000800000000C000C00000000000080
:100563000000000000000006001800600180060083
:1005730018002000000007F0080810041004080801
:1005830007F000000000080408041FFC0004000436
:100593000000000000000E0C1014102410441184FD
:1005A3000E0C000000000C18100411041104128832
:1005B3000C700000000000E00320042408241FFC4A
:1005C3000024000000001F981084110411041088F7
:1005D30010700000000007F0088811041104188847
:1005E3000070000000001C00100010FC13001C0031
:1005F3001000000000000E381144108410841144D0
:100603000E38000000000700088C104410440888CE
:1006130007F00000000000000000030C030C0000C2
:1006230000000000000000000001010600000000BF
:1006330000000000000000800140022004100808B0
:1006430010040000022002200220022002200220C7
:1006530002200000000010040808041002200140DA
:100663000080000000000E001200100C106C1080BF
:100673000F00000003E00C1813E4142417C4082827
:1006830007D000000004003C03C41C40074000E402
:10069300001C000410041FFC1104110411040E8833
:1006A3000070000003E00C1810041004100410087C
:1006B3001C10000010041FFC100410041004080890
:1006C30007F0000010041FFC1104110417C41004E8
:1006D3000818000010041FFC1104110017C01000BB
:1006E3000800000003E00C181004100410441C78E8
:1006F3000040000010041FFC108400800080108460
:100703001FFC10040000100410041FFC100410044C
:100713000000000000030001100110011FFE100083
:100723001000000010041FFC110403801464181C43
:100733001004000010041FFC100400040004000453
:10074300000C000010041FFC1F0000FC1F001FFC16
:100753001004000010041FFC0C04030000E0101838
:100763001FFC100007F00808100410041004080808
:1007730007F0000010041FFC10841080108010800C
:100783000F00000007F0081810241024101C080A9A
:1007930007F2000010041FFC1104110011C01130F6
:1007A3000E0C000400000E1C11041084108410446D
:1007B3001C3800001800100010041FFC1004100067
:1007C3001800000010001FF81004000400041004B7
:1007D3001FF8100010001E0011E0001C00701380B1
:1007E3001C0010001FC0103C00E01F0000E0103C84
:1007F3001FC000001004180C163401C001C01634C9
:10080300180C100410001C00130400FC13041C003B
:10081300100000000804101C1064108413041C044E
:10082300101800000000000000007FFE400240029C
:1008330040020000000030000C0003800060001C38
:100843000003000000004002400240027FFE00005F
:1008530000000000000000002000400040004000B5
:10086300200000000001000100010001000100015F
:1008730000010001000040004000200000000000D3
:1008830000000000000000980124014401440144D9
:1008930000FC000410001FFC008801040104008810
:1008A30000700000000000700088010401040104CE
:1008B3000088000000000070008801040104110892
:1008C3001FFC0004000000F80144014401440144FA
:1008D30000C800000000010401040FFC110411040E
:1008E30011001800000000D601290129012901C9BE
:1008F3000106000010041FFC008401000100010434
:1009030000FC000400000104190419FC00040004A5
:10091300000000000000000300010101190119FE9D
:100923000000000010041FFC0024004001B4010C6F
:10093300010400000000100410041FFC0004000464
:1009430000000000010401FC0104010001FC01049A
:10095300010000FC010401FC00840100010001040A
:1009630000FC0004000000F8010401040104010478
:1009730000F80000010101FF008501040104008863
:1009830000700000000000700088010401040105EC
:1009930001FF00010104010401FC008401040100C2
:1009A30001800000000000CC012401240124012463
:1009B3000198000000000100010007F80104010490
:1009C30000000000010001F8000400040004010815
:1009D30001FC0004010001800170000C00100160A3
:1009E3000180010001F0010C003001C00030010C56
:1009F30001F0010000000104018C00740170018CFE
:100A030001040000010101810171000E0018016061
:100A13000180010000000184010C013401440184C0
:100A2300010C0000000000000000000001003EFC7B
:100A3300400240020000000000000000FFFF000031
:100A4300000000000000400240023EFC01000000E4
:100A530000000000000060008000800040004000B3
:100A63002000200000000000000000000000000043
:100A73000000000000000000000000000000000073
:100A83000000000000000000000000000000000063
:100A9300000000000000000F80380FFE380F803880
:100AA3000000000000000000000000000000000043
:100AB30000000100000600000C00003800003100B7
:100AC300000600000C0000380000300000000000A9
:100AD3000000000061800067F807F9800061800072
:100AE30061800061800061800067F807F980006120
:100AF3008000000000000000000001C0E003E0F0FF
:100B03000630080418081FFFFE040E080787F003C9
:100B130081E000000000000001F000060C00040466
:100B230008060C7001F9C0000E00003BE000EC1851
:100B3300070808040C180003E00000000001E000AF
:100B430007F003F818041C0804170807E1D003C0D2
:100B5300E00023B0003C0800200800001000000063
:100B63000000000100003100003200001C00000002
:100B73000000000000000000000000000000000072
:100B83000000000000000000000000000000000062
:100B9300000000007F0001FFC00780F00C00181068
:100BA30000042000020000000000002000021000EA
:100BB300040C00180780F001FFC0007F0000000054
:100BC3000000000000000000000000000000000022
:100BD3004200006600006600003C0000180003FFAE
:100BE300C0001800003C00006600006600004200E0
:100BF30000000000080000080000080000080000D2
:100C0300080001FFC00008000008000008000008F9
:100C13000000080000000000000100003100003265
:100C230000001C00000000000000000000000000A5
:100C330000000000000000000000000008000008A1
:100C43000000080000080000080000080000080079
:100C53000008000008000008000000000000000079
:100C630000000000380000380000380000000000D9
:100C73000000000000000000000000000000000071
:100C830000000000000600001C000070000180004E
:100C93000E0000380000C0000700001C00003000F8
:100CA30000000000000000007F8001FFE00380706F
:100CB30006001804000804000806001803807001E9
:100CC300FFE0007F80000000000000000000010042
:100CD3000801000801000803FFF807FFF8000008F7
:100CE30000000800000800000000000000000001F0
:100CF300C03802C058040098040118040218040400
:100D030018061C1803F81801E0F8000000000000A2
:100D130000000001C0E003C0F00400080408080458
:100D2300080806180803F41801E7F00001E00000C2
:100D330000000000000000000300000D000011008F
:100D430000610000810803010807FFF80FFFF800A6
:100D530001080001080000000000000000E007FC9B
:100D6300D0060808061008061008061008061838EA
:100D7300060FF00607C0000000000000000000009E
:100D83003F8001FFE00384300208180410080410B8
:100D930008041008071810030FF00007C000000034
:100DA30000000000000003C000070000060000066A
:100DB30000F80607F806180006E000070000060022
:100DC3000000000000000001E1E003F7F00634102A
:100DD300041808041808040C08040C080616180361
:100DE300F3F001C1E000000000000000F80003FC84
:100DF300300306380402080402080402080404103D
:100E03000308F001FFC0007F0000000000000000A5
:100E130000000000000000000000000070380070B7
:100E230038007038000000000000000000000000DF
:100E330000000000000000000000000000000000AF
:100E4300301A00301C000000000000000000000009
:100E53000000000000000000000000080000140073
:100E630000220000410000808001004002002004B5
:100E7300001008000800000000000000210000210D
:100E830000002100002100002100002100002100BA
:100E930000210000210000210000000000000000EC
:100EA3000000080008040010020020010040008038
:100EB3008000410000220000140000080000000030
:100EC30000000003C00004C000040000080038084C
:100ED3000F380808380810000C300007E00003C082
:100EE30000000000000000003F8000FFE00380706E
:100EF300020F1006708804C088048308047F8802E8
:100F0300C09003012000FE4000000800001800010B
:100F1300F8003E0801C20007020007E20000FE00DD
:100F2300001FC80001F8000038000008040008078B
:100F3300FFF807FFF8040808040808040808040871
:100F43000806180803F41801E7F00001E0000000A8
:100F5300000000003F8001FFE003807002001804DE
:100F6300000804000804000804001006002007809D
:100F7300C000000004000807FFF807FFF80400089A
:100F83000400080400080400180200100380700124
:100F9300FFE0007F8000000004000807FFF807FF60
:100FA300F8040808040808040808040808043E08AC
:100FB3000400080600180100600000000400080790
:100FC300FFF807FFF80408080408000408000408F1
:100FD30000043E000600000600000180000000003F
:100FE300000000003F8001FFE0038070060018044A
:100FF30000080402080402080203F00783F0000259
:101003000000020004000807FFF807FFF8040808BF
:101013000008000008000008000008000408080792
:10102300FFF807FFF80400080000000000000400B8
:101033000804000804000807FFF807FFF804000885
:101043000400080400080000000000000000000085
:101053000006000007000001040001040001040071
:101063000307FFFE07FFFC04000004000004000068
:1010730004000807FFF807FFF8040C080018000035
:101083003E0004C7800503C80600F80400380400C6
:101093001800000804000807FFF807FFF804000819
:1010A3000000080000080000080000080000080015
:1010B300001800006000000004000807FFF8078024
:1010C3000807FC00007FC00003F80007C000780099
:1010D30007800807FFF807FFF80400080400080763
:1010E300FFF807000803C00000E000003800001EFE
:1010F300000007000001C00400F007FFF80400002F
:10110300000000007F8001FFE003807006001804E8
:10111300000804000806001803003001FFE0007F08
:101123008000000004000807FFF807FFF804040824
:10113300040400040400040400040400060C000377
:10114300F80001F000000000000000007F8001FFB4
:10115300E00380700600880400880400C806003C91
:1011630003003E01FFE6007F84000000040008073F
:10117300FFF807FFF8040808040800040C00040F34
:1011830000040BC00610F003F03801E0080000086B
:1011930000000001E0F803F03006301004180804E2
:1011A3001808040C08040C080206180207F007814B
:1011B300E0000000018000060000040000040000BD
:1011C30004000807FFF807FFF80400080400000400
:1011D300000006000001800004000007FFE007FF95
:1011E300F0040018000008000008000008000008D0
:1011F30000000804001007FFE004000004000006DC
:10120300000007E00007FE00041FE00001F80000F3
:10121300380001E0043E0007C0000600000400009F
:1012230004000007E00007FFC0041FF80007C00721
:10123300F80007FF80043FF80007C004F800070028
:101243000004000000000004000806001807C0782E
:1012530005F1C8003E00001F800463E80780F8061C
:1012630000180400080000000400000600000780C6
:101273000007E008047C08001FF80007F8001808BE
:1012830004E008070000060000040000000000015D
:1012930000080600380400F80403E8040F08047C7F
:1012A3000805F00807C008070018040060000000E4
:1012B3000000000000000000000000000000003FEC
:1012C300FFFE200002200002200002200002200076
:1012D30002000000000000000000080000070000FA
:1012E30000C0000038000006000001C0000030000C
:1012F300000E0000010000000000000000002000BC
:10130300022000022000022000022000023FFFFE14
:1013130000000000000000000000000000000000CA
:101323000000000000080000100000300000200052
:101333000030000010000008000000000000000062
:101343000000010000010000010000010000010095
:101353000001000001000001000001000001000085
:101363000100000100000000000000000020000058
:10137300200000100000100000000000000000002A
:1013830000000000000000000000000000F0001951
:10139300F8001B1800220800260800240800241067
:1013A300003FF8001FF800000800001800000004C8
:1013B300000007FFF80FFFF00018180010080020C6
:1013C30008002008003018001FF0000FC0000000C4
:1013D3000000000007C0001FF000183000200800C4
:1013E3002008002008003C08001C100000600000DA
:1013F300000000000000000007C0001FF0003818C4
:1014030000200800200800200804101007FFF80F30
:10141300FFF00000100000000000000000000007C3
:10142300C0001FF00012300022180022080022081A
:10143300003208001E10000E200000000000000013
:10144300200000200800200801FFF803FFF8062011
:1014530008042008042008072000030000000000FF
:1014630000000000000E000E6E001FF30031B100FB
:1014730020B10020B1003191001F13002E1E002067
:101483000E00300000000004000807FFF80FFFF80B
:10149300001008002000002000002008003FF80092
:1014A3001FF80000080000000000000000000020FA
:1014B30008002008002008063FF8063FF80000084F
:1014C3000000080000080000000000000000000009
:1014D30000000000030000030020010020010020A1
:1014E30003063FFE063FFC00000000000000000072
:1014F30000000004000807FFF80FFFF80001880050
:101503000300002FC00038F8002038002008000036
:1015130008000000000000000000040008040008A8
:1015230004000807FFF80FFFF80000080000080098
:101533000008000000000000002008003FF8003F02
:10154300F8001008002000003FF8003FF8001008E2
:10155300002000003FF8003FF800000800000000F2
:101563002008003FF8003FF800100800100000209A
:1015730000002008003FF8001FF8000008000000EA
:101583000000000007C0000FF00018300030080012
:101593002008002008003008001830000FF0000772
:1015A300C0000000000000002001003FFF003FFFDB
:1015B3000010110020090020080020080030380026
:1015C3001FF0000FC00000000000000007C0001F54
:1015D300F00038180020080020080020090010112E
:1015E300001FFF003FFF0000010000000020080073
:1015F3002008002008003FF8003FF800080800100A
:101603000800200800200000300000300000000027
:10161300000000000000000C78001E1800330800D2
:1016230023080021080021880021980030F00038A9
:1016330060000000000000002000002000002000E7
:1016430000FFF003FFF80020080020080020080036
:101653000030000000000000000000002000003FF8
:10166300F0007FF8000018000008000008002010B8
:10167300003FF8007FF000001000000000000000B1
:101683002000003000003C00003F800023F00000F9
:1016930078000070002380003C0000300000200030
:1016A300002000003C00003FE00023F80000E000C1
:1016B3002700003E00003FE00021F80001E0003E6B
:1016C3000000200000000000200800200800383837
:1016D300003E680027800003C8002CF8003838005B
:1016E3002018002008000000000000002000003047
:1016F30003003C01003F830023EC000070002380C3
:10170300003C00002000002000000000000000005A
:1017130000000038080020380020F80023E8002FDC
:1017230088003E0800380800201800007000000000
:1017330000000000000000000000000000000000A6
:1017430008000014001FF7FC300006200002000010
:101753000000000000000000000000000000000086
:10176300000000000000FFFFFF0000000000000079
:101773000000000000000000000000000000200046
:10178300023000061FF7FC001400000800000000F0
:10179300000000000000000000000000000000182E
:1017A3000000600000400000400000200000100026
:1017B300000800000400000400000C0000100000FA
:1043DA00481E7C014000F00000FFFF4C1E700000E8
:0A43EA00000000000000001000F0C9
:0E462E00EF1FAC0670011E4C60030080F322EB
:1045D200EF1FAA0670011E4A6012E4FDEDC3940C9F
:0C45E20050EEE4FC0CECB4A6FB0D80F0E5
:0145EE0022AA
:06460800FF12460EAF0593
:10460E00C2B0C2B2C2B17590FF8F90D2B0C2B0220A
:10461E00C2B0D2B2C2B17590FF8F90D2B0C2B022EA
:104593007590FFC2B0D2B2D2B17F017E0012462E17
:0F45A300D2B07F0A7E0012462EAF907E00C2B0CB
:0145B20022E6
:10443F00901DD8FEE0FCA3E0FDC3901DD0E09DFDD4
:0E444F00901DCFE09CFC901DD3E0FAA3E0FB93
:10445D00901DFCEEF0A3EFF012460E901DFCE01245
:10446D004608E4FF12460EAF0312461EEAFF02464F
:01447D001E20
:102DED00901DE4F0A3EFF0901DD3E0FFA3E0901D44
:0E2DFD00E6CFF0A3EFF0901DDCE0FEA3E0FFB8
:0E2E0B00901DDEEEF0A3EFF0A3ECF0A3EDF0CF
:102E1900E4901DEAF0A3F0A3F0A3F0901DDEE0FE1C
:102E2900A3E0FFC3EB9FFFEA9E901DEEF0A3EFF036
:102E3900901DE0E0FAA3E0FBC3901DE5E09BFE9046
:102E49001DE4E09A901DF0F0A3CEF0901DDEE0FFA6
:102E5900A3E0901DF8CFF0A3EFF0A3EAF0A3EBF005
:102E6900901DEEE0FEA3E0FFD39400EE6480948011
:102E7900400A901DF4E4F0A304F08021EF4E70089D
:102E8900901DF4F0A3F0801574FF901DF4F0A3F0E9
:102E9900C3E49FFFE49E901DEEF0A3EFF0901DF0B8
:102EA900E0FEA3E0FFD39400EE64809480400A9092
:102EB9001DF6E4F0A304F08021EF4E7008901DF692
:102EC900F0A3F0801574FF901DF6F0A3F0C3E49F02
:102ED900FFE49E901DF0F0A3EFF0901DF0E0FEA33B
:102EE900E0FF901DEEE0FCA3E0FDD39FEE6480F8C7
:102EF900EC648098901DF24007ECF0A3EDF080059A
:102F0900EEF0A3EFF0E4901DE8F0A3F0901DF3E0DC
:102F19002401FF901DF2E03400FED3901DE9E09FEB
:102F2900901DE8E09E4003022FF8901DF8E0FEA3F3
:102F3900E0FFA3E0FCA3E0FD901DE6124458901DBC
:102F4900EEE0FEA3E0FF901DEBE02FF0901DEAE01C
:102F59003EF0901DF0E0FEA3E0FF901DEDE02FF0A4
:102F6900901DECE03EF0901DF2E0FEA3E0FF901D05
:102F7900EAE0FCA3E0FDD39FEE6480F8EC6480985E
:102F89004020ED9FFFEC9E901DEAF0A3EFF0901D0D
:102F9900F4E0FEA3E0FF901DF9E02FF0901DF8E0AA
:102FA9003EF0901DF2E0FEA3E0FF901DECE0FCA3D3
:102FB900E0FDD39FEE6480F8EC6480984020ED9F9B
:102FC900FFEC9E901DECF0A3EFF0901DF6E0FEA340
:102FD900E0FF901DFBE02FF0901DFAE03EF0901D00
:0F2FE900E9E004F07006901DE8E004F0022F15F7
:012FF80022B6
:103CBE00901DCDEAF0A3EBF0901DC9EEF0A3EFF04E
:103CCE00A3ECF0A3EDF0C007A3E0FAA3E0FB901D78
:103CDE00CBE0FFA3E0901DE4CFF0A3EFF0901E82A7
:103CEE00E0FFA3E0901DE6CFF0A3EFF0D007122E79
:103CFE000B901DC9E0FAA3E0FBFFAE02C007A3E0E4
:103D0E00FCA3E0FD901DCFE0FFA3E0901DE4CFF0FB
:103D1E00A3EFF0901E82E0FFA3E0901DE6CFF0A38C
:103D2E00EFF0D007122E0B901DCFE0FCA3E0FD901C
:103D3E001DCDE0FAA3E0FBA3E0FFA3E0901DE4CFCE
:103D4E00F0A3EFF0901E82E0FFA3E0901DE6CFF00F
:103D5E00A3EFF0901DC9122E06901DCDE0FAA3E040
:103D6E00FBFFAE02C007901DCBE0FCA3E0FD901D53
:103D7E00CFE0FFA3E0901DE4CFF0A3EFF0901E8202
:103D8E00E0FFA3E0901DE6CFF0A3EFF0D007022EE8
:013D9E000B19
:0E2BAC00901EB6EEF0A3EFF0A3ECF0A3EDF058
:102BBA00E4A3F0A3F0EBFF7E00A3EEF0A3EFF02571
:102BCA00E0FFEE33FEC374039F901EBFF0E49E90B5
:102BDA001EBEF0901EBCE0FEA3E0FF901EBAE0FC11
:102BEA00A3E0FDD39FEE6480F8EC64809840030272
:102BFA002DEC901EB7E02DFF901EB6E03CFE901E15
:102C0A00BCE0FCA3E0FDC3901EB9E09DFD901EB898
:102C1A00E09CFC901E82124458901EBCE0FEA3E089
:102C2A00FF901EB7E02FFF901EB6E03EFE901EBA40
:102C3A00E0FCA3E0FDC3901EB9E09DFD901EB8E044
:102C4A009CFC901E82124458901EBCE0FEA3E0FF3A
:102C5A00901EB7E02FFF901EB6E03EFE901EBAE02F
:102C6A00FCA3E0FD901EB9E02DFD901EB8E03CFCEF
:102C7A00901E82124458901EBAE0FEA3E0FF901EF6
:102C8A00B7E02FFF901EB6E03EFE901EBCE0FCA30C
:102C9A00E0FD901EB9E02DFD901EB8E03CFC901EB0
:102CAA0082124458901EBAE0FEA3E0FFC3901EB7FA
:102CBA00E09FFF901EB6E09EFE901EBCE0FCA3E0E3
:102CCA00FD901EB9E02DFD901EB8E03CFC901E82DE
:102CDA00124458901EBCE0FEA3E0FFC3901EB7E06A
:102CEA009FFF901EB6E09EFE901EBAE0FCA3E0FD98
:102CFA00901EB9E02DFD901EB8E03CFC901E821299
:102D0A004458901EBAE0FEA3E0FFC3901EB7E09FAE
:102D1A00FF901EB6E09EFE901EBCE0FCA3E0FDC341
:102D2A00901EB9E09DFD901EB8E09CFC901E821298
:102D3A004458901EBCE0FEA3E0FFC3901EB7E09F7C
:102D4A00FF901EB6E09EFE901EBAE0FCA3E0FDC313
:102D5A00901EB9E09DFD901EB8E09CFC901E821268
:102D6A004458901EBBE004F07006901EBAE004F0CE
:102D7A00C3901EBEE0648094805025901EBAE0FE87
:102D8A00A3E07802C333CE33CED8F92406FFE43E5B
:102D9A00FE901EBFE02FF0901EBEE03EF0022BDD3B
:102DAA00901EBCE0FEA3E0FFC3901EBBE09FFF9015
:102DBA001EBAE09EFEEF7802C333CE33CED8F92492
:102DCA000AFFE43EFE901EBFE02FF0901EBEE03EDA
:102DDA00F0901EBDE024FFF0901EBCE034FFF0022C
:022DEA002BDDDF
:012DEC0022C4
:1017C300901DCDEEF0A3EFF0A3ECF0A3EDF0A3EAB0
:0417D300F0A3EBF0A4
:1017D7004A7003021FF2901DD1E0FEA3E0FF901DA7
:1017E700D6EEF0A3EFF0A3E4F0A304F07C027DC3F0
:1017F7001220400C7DE8122052A3EEF0A3EFF090E8
:101807001DD5E064016003021DF2901DD6E0FEA322
:10181700E0FFD3901DD9E09FEE6480F8901DD8E0DB
:101827006480984003021CA2901DDAE0FCA3E0FD4F
:10183700EF9DEC6480F8EE648098406E901DCEE0DA
:101847002DFF901DCDE03CCF2401CF3400FEC00614
:10185700C007901DD8E0FEA3E0FF901DD0E02FFD4C
:10186700901DCFE03EFC901DD6E0FEA3E0FF901D4B
:10187700CDE0FAA3E02FFBEA3EFA901DD8E0FEA3E5
:10188700E0FF901DCFE0F8A3E02FFFE83E901DE4B6
:10189700F0A3EFF0901DD3E0FFA3E0901DE6CFF09B
:1018A700A3EFF0D007D006122E0B901DDAE0FEA3AF
:1018B700E0FF2401FDE43EFCC3901DCEE09DEC64F7
:1018C70080F8901DCDE0648098500302195CD39096
:1018D7001DD7E09FEE6480F8901DD6E064809840A5
:1018E70074E0FEA3E0FF901DCDE0FCA3E0FD9FEEBA
:1018F7006480F8EC6480985009E4901DDCF0A3F054
:10190700800DC3ED9FFFEC9E901DDCF0A3EFF090E0
:101917001DD8E0FEA3E0FF901DD0E02FFD901DCF66
:10192700E03EFC901DDAE0FEA3E0FF901DCDE0FA5B
:10193700A3E0C39FFFEA9ECF24FFFBEF34FFFA909B
:101947001DD8E0FEA3E0FF901DCFE0F8A3E02FFF36
:10195700E83E122DED901DD8E0FEA3E0FF901DCFCD
:10196700E0FCA3E0FDC39FEE6480F8EC6480985030
:1019770003021A00901DDAE0FEA3E0FFD3901DD703
:10198700E09FEE6480F8901DD6E0648098406A90EE
:101997001DCEE02FFF901DCDE03ECF2401CF3400B8
:1019A700FEC006C007901DD8E0FEA3E0FFC3ED9F71
:1019B700FDEC9EFC901DD6E0FEA3E0FF901DCDE060
:1019C700FAA3E02FFBEA3EFA901DD8E0FEA3E0FF62
:1019D700901DCFE0F8A3E0C39FFFE89E901DE4F0C1
:1019E700A3EFF0901DD3E0FFA3E0901DE6CFF0A397
:1019F700EFF0D007D006122E0B901DDAE0FEA3E021
:101A0700FF2401FDE43EFCC3901DCEE09DEC648005
:101A1700F8901DCDE06480985003021ACA901DD833
:101A2700E0FCA3E0FD901DD0E09DEC6480F8901DE4
:101A3700CFE06480985003021ACAD3901DD7E09F65
:101A4700EE6480F8901DD6E06480984076E0FEA3AF
:101A5700E0FF901DCDE0FCA3E0FD9FEE6480F8EC75
:101A67006480985009E4901DDCF0A3F0800DC3ED6D
:101A77009FFFEC9E901DDCF0A3EFF0901DD8E0FED9
:101A8700A3E0FFC3901DD0E09FFD901DCFE09EFC1B
:101A9700901DDAE0FEA3E0FF901DCDE0FAA3E0C3BE
:101AA7009FFFEA9ECF24FFFBEF34FFFA901DD8E09B
:101AB700FEA3E0FF901DCFE0F8A3E0C39FFFE89EE1
:101AC700122DED901DD6E0FEA3E0FFA3E0B50616AC
:101AD700A3E0B50711A3E0FCA3E0FDEF6D7002EEF4
:101AE7006C6003021B72901DD6E0FEA3E0FF901D01
:101AF700CFE0FCA3E0FDC39FEE6480F8EC64809820
:101B07005009E4901DDCF0A3F0800DC3ED9FFFECBE
:101B17009E901DDCF0A3EFF0901DD8E0FEA3E0FF40
:101B2700901DCEE02FFB901DCDE03EFAAF03FEC027
:101B370006C007901DDCE0FCA3E0FD901DD6E0FE8B
:101B4700A3E0FF901DCFE0F8A3E02FFFE83E901D34
:101B5700E4F0A3EFF0901DD3E0FFA3E0901DE6CFE4
:101B6700F0A3EFF0D007D006122E0B901DD8E0FEA1
:101B7700A3E0FFC3901DCEE09FEE6480F8901DCDDB
:101B8700E06480985003021C3D901DD6E0FCA3E062
:101B9700FDEFB5051BEEB50417901DDAE0FEA3E0D7
:101BA700FF901DD8E06E7003A3E06F6003021C3D39
:101BB700901DD6E0FEA3E0FF901DCFE0FCA3E0FD63
:101BC700C39FEE6480F8EC6480985009E4901DDCB4
:101BD700F0A3F0800DC3ED9FFFEC9E901DDCF0A3FA
:101BE700EFF0901DD8E0FEA3E0FFC3901DCEE09F6D
:101BF700FB901DCDE09EFAAF03FEC006C007901D07
:101C0700DCE0FCA3E0FD901DD6E0FEA3E0FF901D05
:101C1700CFE0F8A3E02FFFE83E901DE4F0A3EFF03C
:101C2700901DD3E0FFA3E0901DE6CFF0A3EFF0D027
:101C370007D006122E0B901DD9E004F07006901DF8
:101C4700D8E004F0901DD8E0FCA3E0FDFFAE04123D
:101C57002040AA06AB07901DD1E0FCA3E0FDFFAE34
:101C670004122040C3EF9BFBEE9AFA901DD6E0FCCE
:101C7700A3E0FD24FFFFEC34FFFE122040D3EB9FCF
:101C8700EE6480F8EA6480984003021811E024FFAC
:101C9700F0901DD6E034FFF0021811901DDAE0FE37
:101CA700A3E0FF901DCEE02FFF901DCDE03ECF2497
:101CB70001CF3400FEC006C007901DCFE0FCA3E0B3
:101CC700FDA3E0FEA3E0FF901DCDE0FAA3E02FFB0C
:101CD700EA3EFAA3E0FFA3E0901DE4CFF0A3EFF004
:101CE700901DD3E0FFA3E0901DE6CFF0A3EFF0D067
:101CF70007D006122E0B901DDBE02401FF901DDAA2
:101D0700E03400FE901DCDE0FCA3E0FDC39FEE6430
:101D170080F8EC648098405A901DD1E0FEA3E0FF64
:101D2700ED9FEE6480F8EC6480985009E4901DDC28
:101D3700F0A3F0800DC3ED9FFFEC9E901DDCF0A398
:101D4700EFF0901DCFE0FCA3E0FD901DDAE0FEA3CD
:101D5700E0FF901DCDE0FAA3E0C39FFFEA9ECF24EA
:101D6700FFFBEF34FFFAA3E0FFA3E0901DE4CF12DF
:101D77002DF0901DD1E0FEA3E0FF901DCFE0FCA366
:101D8700E0FDC39FEE6480F8EC6480985009E4900E
:101D97001DDCF0A3F0800DC3ED9FFFEC9E901DDCD2
:101DA700F0A3EFF0901DCDE0FAA3E0FBFFAE02C079
:101DB70006C007901DDCE0FCA3E0FD901DD1E0FE0E
:101DC700A3E0FF901DCFE0F8A3E02FFFE83E901DB2
:101DD700E4F0A3EFF0901DD3E0FFA3E0901DE6CF62
:101DE700F0A3EFF0D007D006022E0B901DD6E0FE31
:101DF700A3E0FFD3901DD9E09FEE6480F8901DD833
:101E0700E06480984003021F87901DCEE02FFF906B
:101E17001DCDE03EFE901DD8E0FCA3E0FD901DD057
:101E2700E02DFD901DCFE03C124454901DD6E0FEFE
:101E3700A3E0FFC3901DCEE09FFF901DCDE09EFE67
:101E4700901DD8E0FCA3E0FD901DD0E02DFD901D76
:101E5700CFE03C124454901DD6E0FEA3E0FF901D56
:101E6700CEE02FFF901DCDE03E12443F901DD6E0FF
:101E7700FEA3E0FFC3901DCEE09FFF901DCDE09E27
:101E870012443F901DD8E0FEA3E0FF901DD6E06E00
:101E97007003A3E06F7003021F22901DCEE02FFF97
:101EA700901DCDE03EFE901DD6E0FCA3E0FD901D09
:101EB700D0E02DFD901DCFE03C124454901DD8E09A
:101EC700FEA3E0FF901DCEE02FFF901DCDE03E90DA
:101ED7001DD6124442901DD8E0FEA3E0FFC3901D1B
:101EE700CEE09FFF901DCDE09EFE901DD6E0FCA3A7
:101EF700E0FD901DD0E02DFD901DCFE03C12445435
:101F0700901DD8E0FEA3E0FFC3901DCEE09FFF9099
:101F17001DCDE09EFE901DD6124443901DD9E004CE
:101F2700F07006901DD8E004F0901DD8E0FCA3E007
:101F3700FDFFAE04122040AA06AB07901DD1E0FCBE
:101F4700A3E0FDFFAE04122040C3EF9BFBEE9AFA1D
:101F5700901DD6E0FCA3E0FD24FFFFEC34FFFE124A
:101F67002040D3EB9FEE6480F8EA64809840030238
:101F77001DF2E024FFF0901DD6E034FFF0021DF2C1
:101F8700901DD1E0FEA3E0FF901DCEE02FFF901D36
:101F9700CDE03EFE901DCFE0FCA3E0FD124455903E
:101FA7001DD1E0FEA3E0FFC3901DCEE09FFF901D73
:101FB700CDE09EFE901DCFE0FCA3E0FD12445590BE
:101FC7001DCDE0FEA3E0FF901DD1E0FCA3E0FD9056
:101FD7001DD0E02DFD901DCFE03C124454901DCD47
:0B1FE700E0FEA3E0FF901DD112444378
:011FF20022CC
:08435900901DC0EEF0A3EFF08F
:10436100E4FDFCD3901E7FE09D901E7EE09C4039D1
:10437100E4FF12460E124609FF12460EFBFA901E8A
:104381007DE025E0FF901E7CE033FEC3EB9FEA9EBB
:104391005010901DC0A3E0FF12461E0BBB00010A86
:0943A10080DC0DBD00010C80BAA6
:0143AA0022F0
:10451E00AB07AA06901E70EAF0A3EBF0A3ECF0A393
:10452E00EDF0A3EAF0A3EBF0A3ECF0A3EDF012464E
:0A453E000EEE124608E4FF02460EDE
:0E3F1000901DC7EEF0A3EFF0A3ECF0A3EDF0D0
:103F1E00E4901DD3F0A3F0901DC7E0FEA3E0FFC315
:103F2E00EB9FFFEA9ECF2401CF3400901DD3F0A368
:103F3E00EFF0901DC9E0FFA3E0901DD1CFF0A3EFED
:103F4E00F0901DCDE0FEA3E0FF901DD1E0FCA3E0BC
:103F5E00FDD39FEC9E5042901DC7E0FEA3E0FF12E2
:103F6E00451EE4FDFCD3901DD4E09D901DD3E09C36
:103F7E004017901DD0E0FF12461E901DCFE0FF129D
:103F8E00461E0DBD00010C80DC901DD2E004F070C9
:093F9E00B0901DD1E004F080A8F0
:013FA70022F7
:09463C00901E80EEF0A3EFF022C5
:09464500901E82EEF0A3EFF022BA
:10353A00901DD2EEF0A3EFF0901DD6EBF0901DD4C3
:05354A00ECF0A3EDF020
:10354F00901DDBECF0A3EDF0901DD7E0FF131313EC
:10355F00541FFEEF540760047F0180027F00EE2F9F
:10356F00FF901DD7E0C313FEEF8EF0A4901DDDF08A
:10357F00901DD6E024E0F0E4F9901DDDE0FFE9C3F3
:10358F009F4003023698901DD7E0FFB40C12901D98
:10359F00D6E075F00CA42403F582E5F03400801812
:1035AF00EF64106003023698901DD6E075F010A4FA
:1035BF002477F582E5F03404F583E58229F582E47A
:1035CF003583F583E493901DD9F0E4901DDAF090E4
:1035DF001DD9E030E713901DD2E0FEA3E0FFA3E07A
:1035EF00FCA3E0FD901E828017901DD8E070149010
:1035FF001DD2E0FEA3E0FFA3E0FCA3E0FD901E8040
:10360F00124458901DD9E025E0F0901DD5E004F04C
:10361F007006901DD4E004F0901E7EE0FEA3E0FF44
:10362F00901DD4E0FCA3E0FDC39FEC9E505B901D6A
:10363F00DBE0FEA3E0FFC3ED9FFDEC9EFC901DD7EA
:10364F00E07A00B50530EAB5042C901DD4EEF0A356
:10365F00EFF0901DD3E004F07006901DD2E004F05F
:10366F00901E7CE0FEA3E0FFC3901DD3E09F901D52
:10367F00D2E09E401022901DDAE004F0E0C39408DF
:09368F0050030235DE0902358802
:01369800220F
:10338600901DC1EEF0A3EFF0A3ECF0A3EDF0A3EADD
:04339600F0A3EBF0C5
:10339A00901E70E0FFA3E0901DCECFF0A3EFF09057
:1033AA001E72E0FFA3E0901DD0CFF0A3EFF0901DB6
:1033BA00C9E0FBA3E0FAA3E0F91220157003023575
:1033CA001BB40A40901DCCE0FF901E73E02FF090D2
:1033DA001E72E03400F0E0FEA3E0FF901DD0EEF094
:1033EA00A3EFF0901DCEE0FDA3E0901DC1CDF0A3A8
:1033FA00EDF0A3EEF0A3EFF0901DCAE475F0011210
:10340A00208880AA901DC5E0FEA3E0FF901DCFE0B2
:10341A002FFF901DCEE03EFE901DCCE0FDC313FBB6
:10342A00C3EF9BFFEE9400FED3901DC2E09F901D58
:10343A00C1E09E401EEDFF901DC4E02FF0901DC319
:10344A00E03400F0901DCEE0FFA3E0901DC1CFF064
:10345A00A3EFF0901DC7E0FEA3E0FF901DD1E02F7F
:10346A00FF901DD0E03EFE901DCCE0FDC3EF9DFF16
:10347A00EE9400FED3901DC4E09F901DC3E09E40D1
:10348A000302351B901DC9E0FBA3E0FAA3E0F91281
:10349A002015B40D2B901DCCE0FF901DC4E02FF039
:1034AA00901DC3E03400F0901DCEE0FFA3E0901D14
:1034BA00C1CFF0A3EFF0901DCAE475F00112208885
:1034CA00901DC1E0FEA3E0FFA3E0FCA3E0FD901D78
:1034DA00C9E0FBA3E0FAA3E0F9122015FB901DCC8A
:1034EA00E0901DD7F0901DCDE0901DD8F012353A2E
:1034FA00901DCAE475F001122088901DCCE0C31318
:10350A00FF901DC2E02FF0901DC1E03400F002339D
:10351A00B8901DC1E0FFA3E0901E74CFF0A3EFF0B6
:0F352A00901DC3E0FFA3E0901E76CFF0A3EFF05B
:01353900226F
:0B3D9F00901DFEEBF0A3EAF0A3E9F09A
:103DAA00901DC112228800000064E4FF1241C090F5
:103DBA001E2CEBF0A3EAF0A3E9F04A7003023E6B73
:103DCA00901E297401F0A3741EF0A37401F0901DD3
:103DDA00FEE0F9A3E0FAA3E0901EC8C9F0A3EAF056
:103DEA00A3E9F0901E29E0F9A3E0FAA3E0901ECB24
:103DFA00C9F0A3EAF0A3E9F0901E2CE0FBA3E0FAD5
:103E0A00A3E0F91243F5901E74E0FEA3E0FFA3E0DD
:103E1A00FCA3E0FD901E79E0FB901DC7E4F0A3EB44
:103E2A00F0901E2CE0F9A3E0FAA3E0901DC9C9F0B6
:103E3A00A3EAF0A3E9F0901E79E0901DCCF0901E61
:103E4A0078E0901DCDF0901E7AE0FAA3E0FB1233E1
:103E5A0086901E2CE0FBA3E0FAA3E0F9E4FF1241EE
:013E6A004710
:013E6B002234
:10456F00D2B3C2B4D2B4E4FF30B5010FE4FEC2B38C
:10457F00D2B3EF25E0FF30B5034401FF0EEEB407D1
:03458F00EDC2B3C7
:014592002206
:104047000245EFE493A3F8E493A34003F68001F25B
:1040570008DFF48029E493A3F85407240CC8C3337A
:10406700C4540F4420C8834004F456800146F6DF49
:10407700E4800B01020408102040809043ABE47EEB
:10408700019360BCA3FF543F30E509541FFEE4933E
:10409700A360010ECF54C025E060A840B8E493A305
:1040A700FAE493A3F8E493A3C8C582C8CAC583CA30
:1040B700F0A3C8C582C8CAC583CADFE9DEE780BEE8
:0143F40000C8
:101FF300C2D530F707B2D563F0FF05F030E70CB276
:10200300D5F4048463F0FF05F080018430D502F435
:022013000422A5
:10201500BB010689828A83E0225002E722BBFE02C9
:09202500E32289828A83E49322FC
:10202E00BB010689828A83F0225002F722BBFE0191
:02203E00F3228B
:10204000EF8DF0A4A8F0CF8CF0A428CE8DF0A42EB4
:02205000FE226E
:10205200C2D5EC30E709B2D5E4C39DFDE49CFCEEA9
:1020620030E715B2D5E4C39FFFE49EFE1222BFC340
:10207200E49DFDE49CFC80031222BF30D507C3E43B
:062082009FFFE49EFE2218
:10208800C5F0F8A3E028F0C5F0F8E58215827002E3
:062098001583E038F02280
:10209E00A3F8E0C5F025F0F0E582158270021583F5
:0620AE00E0C838F0E82252
:1020B400BB0110E58229F582E5833AF583E0F5F06A
:1020C400A3E0225009E92582F886F008E622BBFE47
:1020D4000AE92582F8E2F5F008E222E5832AF5838D
:0820E400E993F5F0A3E9932252
:1020EC00F8BB0111E58229F582E5833AF583E8F026
:1020FC00E5F0A3F0225009E92582C8F608A6F022E3
:0D210C00BBFE09E92582C8F2E5F008F222C9
:10211900E88FF0A4CC8BF0A42CFCE98EF0A42CFC65
:102129008AF0EDA42CFCEA8EF0A4CDA8F08BF0A4E3
:102139002DCC3825F0FDE98FF0A42CCD35F0FCEB42
:102149008EF0A4FEA9F0EB8FF0A4CFC5F02ECD3907
:0F215900FEE43CFCEAA42DCE35F0FDE43CFC2274
:1021680075F008758200EF2FFFEE33FECD33CDCC2E
:1021780033CCC58233C5829BED9AEC99E5829840B1
:102188000CF582EE9BFEED9AFDEC99FC0FD5F0D68E
:10219800E4CEFBE4CDFAE4CCF9A88222B800C1B9B8
:1021A8000059BA002DEC8BF084CFCECDFCE5F0CBF6
:1021B800F97818EF2FFFEE33FEED33FDEC33FCEB2F
:1021C80033FB10D703994004EB99FB0FD8E5E4F9EA
:1021D800FA227818EF2FFFEE33FEED33FDEC33FCD7
:1021E800C933C910D7059BE99A4007EC9BFCE99ACB
:1021F800F90FD8E0E4C9FAE4CCFB2275F010EF2F10
:10220800FFEE33FEED33FDCC33CCC833C810D7070F
:102218009BEC9AE899400AED9BFDEC9AFCE899F84A
:0E2228000FD5F0DAE4CDFBE4CCFAE4C8F922DD
:10223600EB9FF5F0EA9E42F0E99D42F0E89C45F0FE
:012246002275
:102247007401FF3395E0FEFDFCA3A3A3E0CF2FF0BD
:10225700E582158270021583E0CE3EF0E582158295
:1022670070021583E0CD3DF0E5821582700215837B
:05227700E0CC3CF02268
:0C227C00ECF0A3EDF0A3EEF0A3EFF022D5
:10228800A8828583F0D083D08212229F12229F12C7
:10229800229F12229FE473E493A3C583C5F0C583EC
:1022A800C8C582C8F0A3C583C5F0C583C8C582C8A0
:0122B8002203
:0622B9008A838982E473B0
:1043F500901EC8E0FFA3E0FEA3E0CF901E32F0A31D
:10440500EEF0A3EFF0901ECBE0CBF0A3E0CAF0A353
:10441500E0C9F07F22901E35AD82AC831220158D48
:10442500828C83F0A309E970010ADFEC901ECBE0D2
:0A443500FBA3E0FAA3E0F90223EC78
:1022BF00BC000BBE0029EF8DF084FFADF022E4CC03
:1022CF00F875F008EF2FFFEE33FEEC33FCEE9DECCC
:1022DF00984005FCEE9DFE0FD5F0E9E4CEFD22ED12
:1022EF00F8F5F0EE8420D21CFEADF075F008EF2F5C
:1022FF00FFED33FD4007985006D5F0F222C398FD4D
:05230F000FD5F0EA22E9
:10238700E5082432F582E4341EF583E0050822903F
:102397001E2F300703901E32E475F001122341020D
:1023A70020152000E97F2ED2008018EF540F2490CB
:1023B700D43440D4FF30040BEF24BFB41A005003C9
:1023C7002461FFE50960021509050CE50C7002059B
:1023D7000B30070E901E2FE475F001122341EF0218
:1023E700202E0245487403D2078003E4C207F5088C
:1023F700901E2F122358E4F509F50BF50CE509603B
:10240700077F201223CA80F5750AFFC201C200C2E6
:1024170002C203C205C206C208122396FF700D301E
:1024270007057F001223DBAF0CAE0B22B4255FC27A
:10243700D5C204122396FF24D0B40A00501A75F0AF
:102447000A780930D50508B6FF0106C6A426F62086
:10245700D5047002D20380D924CFB41A00EF5004F8
:10246700C2E5D2040225DCD20180C6D20080C0D2E8
:102477000280BCD2D580BAD20580B47F201223CA8D
:102487002002077401B5090040F1122387FF1223C8
:10249700CA022404D208D2068095122387FB12238E
:1024A70087FA122387F94A4B700679AD7A267BFFA4
:1024B70020022EE509602A7E008E82758300122392
:1024C7001460060EEE650A70F0C2D5EBC0E0EAC0F4
:1024D700E0E9C0E0EE122623D0E0F9D0E0FAD0E040
:1024E700FB122015FF60AAEBC0E0EAC0E0E9C0E0FC
:1024F7001223CAD0E02401F9D0E03400FAD0E0FB7F
:10250700E50A0460DCD50AD980877BFF7A26791F24
:10251700D202809C791080027908C206C20880081E
:10252700D2D5790A8004790AC2D5E50A047002F582
:102537000AE4FAFDFEFF122387FC7B082001131231
:102547002387FD7B1030000A122387FE122387FFA3
:102557007B20EC3382D592D55013C3E43000069F1D
:10256700FFE49EFEE42001039DFDE49CFCE4CBF820
:10257700C201EC700CCFCECDCCE824F8F870F38014
:1025870017C3EF33FFEE33FEED33FDEC33FCEB33D4
:10259700FB994002FB0FD8E9EB300105F8D0E0C406
:1025A70048B201C0E00AEC4D4E4F78207B0070C264
:1025B700EAB50A0040BCC0E0122625D0F0D0E020E2
:1025C7000104C4C0E0C4B201C0F01223B3D0F0D5F7
:1025D700F0EB02240412236124A153251B58247213
:1025E7004C246E42251F4F2527442527492487431E
:0825F700252D55251146251183
:1025FF004525114726CD5024762D247A2E249D2B48
:10260F00247E23249B2026B62A24364800002495B6
:10261F003F3F3F00790AA2D5200314300509B910B6
:10262F00020404B9080104A2D520060250010420B7
:10263F0002689202B509005034C0E07F20300319C0
:10264F007F30A20272067205500F12267CC202C2A0
:10265F0006C205C2087F30800F300503E9C0E012C3
:10266F0023CA300503D0E0F9D0E0B509CC30051707
:10267F007F30B9100C1223CA7F583004077F78803F
:10268F0003B908031223CA3002057F2D0223CA7F24
:10269F00202008F87F2B2006F322920280CF286E8D
:1026AF00756C6C2900D2011223873001F8C20178B2
:1026BF000930D50108F60224362D5043495812230C
:1026CF00872403B405004001E49026C8931223BB6E
:0D26DF00743A1223BBD20375090402251BB7
:10231400BB010CE58229F582E5833AF583E022507E
:1023240006E92582F8E622BBFE06E92582F8E222C8
:0D233400E58229F582E5833AF583E49322E2
:10234100F8E0FBA3A3E0F925F0F0E5821582700225
:072351001583E0FA38F022C9
:09235800EBF0A3EAF0A3E9F02286
:10236100D083D082F8E4937012740193700DA3A30B
:1023710093F8740193F5828883E47374029368601F
:06238100EFA3A3A380DF1F
:10454800EFB40A07740D124553740A309811A899EC
:10455800B8130CC2983098FDA899C298B811F630D3
:0745680099FDC299F59922AB
:00000001FF
